:0200000480007A
:100000006F00C0006F20802C6F20402C93000000F8
:10001000130100009301000013020000930200008E
:100020001303000093030000130400009304000076
:10003000130500009305000013060000930600005E
:100040001307000093070000130800009308000046
:100050001309000093090000130A0000930A00002E
:10006000130B0000930B0000130C0000930C000016
:10007000130D0000930D0000130E0000930E0000FE
:10008000130F0000930F000097020000938202F804
:100090007390523017A100001301C1E4F32240F124
:1000A0009392C2003301510073100134EF20900B82
:1000B000173500001305858B6F20006B8332851088
:1000C000739012148330850003310501833185015B
:1000D000033205028332850203330503833385032C
:1000E000033405048334850483358505033605060A
:1000F00083368506033705078337850703380508E8
:10010000833885080339050983398509033A050AC7
:10011000833A850A033B050B833B850B033C050CA7
:10012000833C850C033D050D833D850D033E050E87
:10013000833E850E033F050F833F850F033505057D
:10014000730020107311011423341100233C31007B
:10015000233041022334510223386102233C7102CF
:1001600023308104233491042338A104233CB104B7
:100170002330C1062334D1062338E106233CF1069F
:10018000233001092334110923382109233C310983
:100190002330410B2334510B2338610B233C710B6B
:1001A0002330810D2334910D2338A10D233CB10D53
:1001B0002330C10F2334D10F2338E10F233CF10F3B
:1001C000F312011423385100F32200102330511090
:1001D000F322101423345110F32230142338511019
:1001E000F3222014233C5110130501006F208033AB
:1010000000000000000000000000000000000000E0
:1010100000000000000000000000000000000000D0
:1010200000000000000000000000000000000000C0
:1010300000000000000000000000000000000000B0
:081040000000000000000000A8
:10200000B367B500B3E7C70093F77700B306C50021
:10201000638407023386C50093070500637ED502FB
:1020200003C705009385150093871700A38FE7FE6C
:10203000E398C5FE67800000E37ED5FE93070500A8
:1020400003B70500938787009385850023BCE7FECF
:10205000E3E8D7FE6780000067800000130101FFFE
:10206000B367C500233081002334110093F7770054
:10207000130405003307C500638207026376E50099
:1020800093F5F50FEFF09FFD8330810013050400F9
:1020900003340100130101016780000093F5F50F7F
:1020A00093968500B3E6B60093970601B3E7D70091
:1020B00093960702B3E6F600E378E5FC9307050084
:1020C0009387870023BCD7FEE3ECE7FE83308100D3
:1020D00013050400033401001301010167800000AF
:1020E00083470500638E07009307050003C71700A9
:1020F00093871700E31C07FE3385A7406780000025
:1021000013050000678000008347050093851500D4
:102110001305150003C7F5FF638A0700E386E7FE92
:102120001B8507003B05E5406780000013050000A4
:102130006FF05FFFB367B50093F77700639E070208
:10214000137886FF330805016378050393070500BC
:102150006F000001938787009385850063F807016E
:1021600083B6070003B70500E386E6FE3385A74084
:102170003306A640138507003386C5006F00400173
:1021800003C705008347F5FF93851500639AE700B1
:1021900013051500E396C5FE1305000067800000D7
:1021A0003B85E740678000009307050003C70500F3
:1021B0009387170093851500A38FE7FEE31807FEAA
:1021C000678000000347050093060002930705009F
:1021D0006318D70003C7170093871700E30CD7FED7
:1021E0009306D0026300D7069306B0026300D704BB
:1021F00083C60700930500006382060413050000F0
:1022000093871700131725001B8606FD83C607005A
:102210003307A700131717003305E600E39206FE05
:10222000638005023305A0406780000083C6170065
:102230009305000093871700E39206FC1305000046
:102240006780000083C6170093051000938717006E
:10225000E39606FA130500006FF09FFE8347050022
:10226000638007049305101017F7FFFF130787D942
:10227000939505030336070013051500B3E6B70071
:10228000630A060097F7FFFF23BE07DA83370700CC
:10229000E39A07FE2330D70083470500E39C07FC41
:1022A0006780000017F7FFFF1307C7D583370700C4
:1022B000638A070097F7FFFF23B607D88337070025
:1022C000E39A07FE2330A7006F000000130101FF0F
:1022D0001305903423341100EFF0DFFC130101FEED
:1022E0001306810093077101130890006F008000AE
:1022F000930707009376F500138706009305000304
:102300006374D800930570053B07B7002380E7008E
:10231000135545001387F7FFE31CF6FC8347810044
:10232000230C0100638207041305101093060600B6
:1023300017F7FFFF130707CD1315050383350700B4
:102340009386160033E6A700638A050097F7FFFF20
:1023500023BA07CE83370700E39A07FE83C7060038
:102360002330C700E39C07FC1301010267800000D3
:10237000130101FF37F8FFFF233411003307050174
:10238000B7E703006378F7141357C5009306076097
:1023900017360000130606C793973600B307F600FA
:1023A00083B70700337505016390070E977500002A
:1023B0009385C5C503B805006302081483378800F8
:1023C0009778000083B808C423B0F500638E170F18
:1023D0008337080093983600B308160193D7C700D7
:1023E0009397A70013E3F70D93E5F70123B0680077
:1023F00073000512972700009387C7C01317470083
:10240000B387E70003B7070063140710033708001A
:10241000B708040023B0E7000337880023B4E700BF
:10242000F3A80810B707E0FFB307F500371800005E
:10243000130705003388070103BF070083BE870029
:1024400003BE070103B387012330E7012334D7011B
:102450002338C701233C670093870702130707024D
:10246000E39C07FD7390081093973600B306F600BF
:1024700023B0B600730005120F10000083308100F6
:10248000130101016780000013F70704630A0702C4
:1024900013F70708631A07041307F00093E7070808
:1024A0006394E50493963600B306D60023B0F60095
:1024B0007300051283308100130101016780000061
:1024C00093E707046FF01FFE9777000023BC07B265
:1024D0006FF01FF01715000013054598EFF01FD897
:1024E00013053000EFF01FDC171500001305859B66
:1024F000EFF0DFD613053000EFF0DFDA171500003C
:102500001305C59EEFF09FD513053000EFF09FD95E
:10251000171500001305059FEFF05FD41305300079
:10252000EFF05FD883358511130101F82338810658
:10253000233C11062334910623302107233C310527
:10254000233841052334510523306105233C7103B1
:1025500023388103233491032330A103233CB101A9
:102560009307800013040500638AF50E930720008B
:102570006380F506938745FF130710006376F70025
:102580009307F0006392F51A03350411EFF05FDE54
:102590001305040003340107833081078334810667
:1025A0000339010683398105033A0105833A810421
:1025B000033B0104833B8103033C0103833C810211
:1025C000033D0102833D8101130101086FD01FAF5C
:1025D000033785109377370063980706EF0780006D
:1025E000731030000327070083A70700630AF7046E
:1025F0001305101093071004971600009386869415
:1026000017F7FFFF130707A013150503833507000E
:102610009386160033E6A700638A050097F7FFFF4D
:1026200023B207A283370700E39A07FE83C7060099
:102630002330C700E39C07FC13053000EFF09FC672
:1026400013051000EFF01FC617150000130585993C
:10265000EFF0DFC013053000EFF0DFC403290505FC
:10266000371C0000972400009384C499973B000016
:10267000938B4B99370B0400B70AE0FF977D00005E
:10268000938D4D98177A0000130A4A98B7F9030002
:102690006F0080012334F70023B0FD00B71700005E
:1026A000330CFC00630E3C0B9357CC001394470093
:1026B0003387840003370700E30207FE9387076030
:1026C00093973700B387FB0083BC070093F70C0494
:1026D000638E0706732D0B1037160000B3055C01DF
:1026E00013050C002334B100EFF0DFA4630E0500E6
:1026F00093FC0C088335810063800C0437160000BE
:1027000013050C00EFF0DF8FB387840073100D10FA
:1027100003B70D0023B00700E31E07F623B0FD004A
:102720002330FA006FF09FF7171500001305058E90
:10273000EFF0DFB26FF05FF01715000013050587AB
:10274000EFF0DFB113053000EFF0DFB51715000033
:1027500013054582EFF09FB013053000EFF09FB4F2
:1027600013050900EFF01FB4F32740F1639A07182F
:102770009757000093870789130101ED93D7C7008E
:1027800023308112176800001308C887130405005E
:102790009397A700174500001305C586233411122F
:1027A0009356C5001357C80093E7170097380000E9
:1027B000938848851306F0FF233CF5FE9396A60008
:1027C0001317A700B707002093E61600136717003A
:1027D00093D5C8001313F6039387F70C233CF8FE38
:1027E00023B0D8002330E500B3E7650073900718E5
:1027F00073270018639EE7141356B6009307F00181
:102800009702000093824201F39252307310063B0C
:102810007390073A739052301308F0BF13185801A1
:1028200097E7FFFF93874792B3870701739057108D
:10283000F3270034B387070173900714B7B700007C
:102840009B87071073902730B7E701009B870760CD
:10285000739007307350403017270000130787B973
:102860009307083EB3060701B307F700B70808004F
:1028700017660000233CD67817230000130383F665
:102880009766000023B0F6789388F8039307500208
:102890001308080113D61700B3861701B347F600D3
:1028A000B30507019396C600939757002330D700CE
:1028B0002334B70093F7070213070701B367F60045
:1028C000E31AE3FC13060012930500001305010050
:1028D0009727000023B407F0EFF04FF8B707008008
:1028E0003304F4001305010023348110EFD00FFDF1
:1028F0008330811203340112130101136780000039
:1029000013071000B7B7130937060800938727A7E6
:102910001306C6FF1315F7019316E7036F00C001F6
:102920002F20070013D71700B3C7E7009397E703DB
:10293000B3F7D700B3E7E70033F7C70093F5170005
:102940003307A700E39E05FC032007006FF09FFDFF
:10295000170500001305856EEFF05F90130530003A
:10296000EFF05F9467800000930000001301000007
:10297000338720409303000093012000631E774AB1
:1029800093001000130110003387204093030000D0
:10299000930130006312774A9300300013017000F6
:1029A000338720409303C0FF9301400063167748AC
:1029B000930000003781FFFF33872040B78300007A
:1029C00093015000631A7746B7000080130100009E
:1029D00033872040B703008093016000631E774473
:1029E000B70000803781FFFF33872040B783008026
:1029F0009301700063127744930000003781000058
:102A00001B01F1FF33872040B783FFFF9B83130037
:102A10009301800063127742B70000809B80F0FF33
:102A20001301000033872040B70300809B83F3FF2E
:102A30009301900063127740B70000809B80F0FF05
:102A4000378100001B01F1FF33872040B783FF7FF0
:102A50009301A0006312773EB70000803781000029
:102A60001B01F1FF33872040B703FFFF9B83F3FF78
:102A70009393F300938313009301B000631E773A9E
:102A8000B70000809B80F0FF3781FFFF3387204035
:102A9000B70301009B8313009393F3009383F3FF29
:102AA0009301C000631A7738930000001301F0FF10
:102AB00033872040930310009301D000631E7736C4
:102AC0009300F0FF13011000338720409303E0FFD1
:102AD0009301E000631277369300F0FF1301F0FFDB
:102AE00033872040930300009301F000631677348E
:102AF0009300D0001301B000B38020409303200066
:102B000093010001639A70329300E0001301B0005A
:102B1000338120409303300093011001631E713014
:102B20009300D000B3801040930300009301200174
:102B300063947030130200009300D0001301B000C2
:102B40003387204013030700130212009302200072
:102B5000E31452FE9303200093013001631E732C93
:102B6000130200009300E0001301B00033872040FF
:102B70001300000013030700130212009302200049
:102B8000E31252FE93033000930140016316732A4F
:102B9000130200009300F0001301B00033872040BF
:102BA00013000000130000001303070013021200BB
:102BB00093022000E31052FE930340009301500162
:102BC000631C7326130200009300D0001301B000B1
:102BD000338720401302120093022000E31652FEB6
:102BE000930320009301600163187724130200000F
:102BF0009300E0001301B000130000003387204071
:102C00001302120093022000E31452FE93033000DB
:102C10009301700163127722130200009300F00009
:102C20001301B000130000001300000033872040A0
:102C30001302120093022000E31252FE930340009D
:102C400093018001631A771E130200009300D000E5
:102C5000130000001301B00033872040130212005C
:102C600093022000E31452FE93032000930190018D
:102C70006314771C130200009300E00013000000AF
:102C80001301B0001300000033872040130212002C
:102C900093022000E31252FE930330009301A0013F
:102CA000631C7718130200009300F000130000006B
:102CB000130000001301B0003387204013021200FC
:102CC00093022000E31252FE930340009301B001EF
:102CD00063147716130200001301B0009300D000B4
:102CE000338720401302120093022000E31652FEA5
:102CF000930320009301C0016310771413020000B6
:102D00001301B0009300E00013000000338720405F
:102D10001302120093022000E31452FE93033000CA
:102D20009301D001631A7710130200001301B00061
:102D30009300F000130000001300000033872040D0
:102D40001302120093022000E31252FE930340008C
:102D50009301E0016312770E130200001301B0002B
:102D6000130000009300D0003387204013021200AC
:102D700093022000E31452FE930320009301F0011C
:102D8000631C770A130200001301B0001300000057
:102D90009300E0001300000033872040130212006C
:102DA00093022000E31252FE9303300093010002CD
:102DB00063147708130200001301B0001300000031
:102DC000130000009300F00033872040130212002C
:102DD00093022000E31252FE93034000930110027D
:102DE000631C7704930010FF330110409303F0003D
:102DF00093012002631271049300000233810040AA
:102E0000930300029301300263187102B300004083
:102E1000930300009301400263907002930000014D
:102E20001301E0013380204093030000930150021E
:102E300063147000631A30001395110063000500DD
:102E400013651500730000001305100073000000E7
:042E5000731000C03B
:102E5800417373657274696F6E206661696C65642D
:102E68003A2061646472203E3D202831554C203C54
:102E78003C203132292026262061646472203C20BF
:102E88003633202A202831554C203C3C2031322929
:102E98000A00000000000000417373657274696FD6
:102EA8006E206661696C65643A20212870745B3312
:102EB8005D5B616464722F2831554C203C3C2031A5
:102EC80032295D20262030783038302920262620E7
:102ED8006361757365203D3D203078660A00000007
:102EE800417373657274696F6E206661696C65649D
:102EF8003A206E6F64650A00417373657274696F76
:102F08006E206661696C65643A20757365725F6DE1
:102F1800617070696E675B616464722F2831554C0B
:102F2800203C3C203132295D2E61646472203D3D95
:102F380020300A0000000000417373657274696FE5
:102F48006E206661696C65643A202122696C6C6543
:102F580067616C20696E737472756374696F6E2231
:102F68000A00000000000000417373657274696F05
:102F78006E206661696C65643A2070745B335D5BD2
:102F8800616464722F2831554C203C3C2031322931
:102F98005D20262030783034300A00000000000020
:102FA800417373657274696F6E206661696C6564DC
:102FB8003A2070745B335D5B616464722F2831550D
:102FC8004C203C3C203132295D2026203078303896
:102FD800300A000000000000417373657274696F65
:102FE8006E206661696C65643A2074662D3E657072
:102FF8006320252034203D3D20300A0000000000D9
:10300800417373657274696F6E206661696C65647B
:103018003A202122756E6578706563746564206551
:103028007863657074696F6E220A00000000000002
:10303800417373657274696F6E206661696C65644B
:103048003A202122756E737570706F7274656420F2
:0C30580073617470206D6F6465220A00C3
:040000058000000077
:00000001FF
